:100000001F306500003066000030860000309F0021
:100010000030A00020308E0032308F00043090007D
:100020002C3093004D309800683099007A309A0057
:1000300020309B00A030A6000030A700F522051E4E
:10004000242852309C002B2854309C000A309D00FC
:100050006F204D232F2800309D006F204D239423C7
:100060002F22051E442800309D006F204D23523062
:100070009C009423B322051E4428851D5328051C8B
:100080006028851C5B283B280A309D0054309C006A
:100090009423B322051A3328851D5728051C6A2886
:1000A000851C65284A2800309D00AD203B280A3079
:1000B0009D00AD204A283F214D23E221B3223B2859
:1000C000E3204D239B21B3223B286D214D23E221C8
:1000D000B3224A2811214D239B21B3224A281D080F
:1000E00089008316081483120808AA00890A831657
:1000F000081483120808A900890A831608148312B9
:100100000808A800890A83160814831208089000BA
:10011000890A83160814831208089100890A831635
:100120000814831208089200890A8316081483129F
:1001300008089400890A8316081483120808950099
:10014000890A83160814831208089600890A831600
:10015000081483120808970008001D0889002A085F
:100160008800D720890A29088800D720890A28080A
:100170008800D720890A10088800D720890A11082A
:100180008800D720890A12088800D720890A140815
:100190008800D720890A15088800D720890A160800
:1001A0008800D720890A17088800D72008008316FE
:1001B000081555308900AA3089008814081EDE28E9
:1001C00008128312080000308C00051DEA289423D1
:1001D0009423EB289D2302302A020319F0280329D7
:1001E000173029020319F528032930302802031992
:1001F000FA2803293030A8001730A9000230AA00DD
:1002000001308C001029A80A281B0729102900306A
:10021000A800A90A0030290203190F291029AA0AE7
:10022000080000308C00051D1829942394231929F7
:100230009D2306302A0203191E293129393029024B
:10024000031923293129303028020319282931299B
:100250003030A8003930A9000630AA0001308C00E7
:100260003E29A80A281B35293E290030A800A90AE2
:100270000030290203193D293E29AA0A080000304E
:100280008D00051D46299423942347299D2306307C
:100290002A0203194C295F293930290203195129EF
:1002A0005F2930302802031956295F293030A80011
:1002B0003930A9000630AA0001308D006C29A8034E
:1002C000A81B63296C293F30A800A903FF3029022D
:1002D00003196B296C29AA03080000308D00051D45
:1002E00074299423942375299D2305302A02031928
:1002F0007A298D299D30290203197F298D292030E3
:100300002802031984298D292030A8009D30A900D6
:100310000530AA0001308D009A29A803A81B912955
:100320009A293F30A800A903FF302902031999290F
:100330009A29AA03080001300C02031DA029080015
:1003400000301502031DAB290230950005309600E0
:1003500000309700080002301502031DB629053051
:100360009500003096000030970008000530150217
:10037000031DC12907309500053096000030970015
:10038000080007301502031DE129003095000030F8
:10039000960000309700940A0A301402031DE129E8
:1003A00000309400920A0A301202031DE129003045
:1003B0009200910A0A301102031DE12900309100D8
:1003C000900A080001300D02031DE72908000730DC
:1003D0001502031DF229053095000030960000300B
:1003E0009700080005301502031DFD290230950015
:1003F0000530960000309700080002301502031DFA
:10040000082A003095000030960000309700080060
:1004100000301502031D2E2A073095000530960086
:10042000003097009403FF301402031D2E2A093078
:1004300094009203FF301202031D2E2A093092000D
:100440009103FF301102031D2E2A09309100900301
:10045000FF301002031D2E2A0930900008000030E2
:100460008600003066008B2386108B233030860098
:10047000000086158B238B23861186100000000058
:10048000203086000000000086158B2386110000B6
:100490000000861000002830A4006F2200008610A3
:1004A00000000830A4006F22000086100000063013
:1004B000A40000006F220000861000000C30A40091
:1004C00000006F220000061100008610000082303C
:1004D000A40000006F220000861400000800861CA3
:1004E0002510861825148610000006150000F0302F
:1004F00066000000861500000608A20000008611B4
:10050000000000008615000000008611A21B7A2A58
:100510000000251C86102518861400000611000016
:100520000030660000002408A30000000F3086059C
:100530000000F030A40500002408860400008615A1
:10054000000086110000A30E00000F308605000099
:10055000F030A30500002308860400008615000083
:1005600086110000080086108030A4006F228614D7
:100570002030A4006F223230A4006F221008303ED9
:10058000A4006F221108303EA4006F221208303EF2
:10059000A4006F221308A4006F221408303EA400A8
:1005A0006F221508303EA4006F228610C030A400D0
:1005B0006F2286141608303EA4006F221708303EC2
:1005C000A4006F221808A4006F221908A4006F224B
:1005D0001A08A4006F222030A4006F221C08A40077
:1005E0006F225830A4006F22080006150000861400
:1005F000000086100000061100000000000000004E
:1006000006110000861400008610000000000000A3
:100610000000061500008614000086100000061178
:100620000000000000000000061100008614000019
:100630008610000000000000000006309E00270821
:10064000A200A21F0611A21B061586140000861028
:100650000000A20D9E0B212B08309E002608A20050
:10066000A21F0611A21B06158614000086100000AA
:10067000A20D9E0B302B0000000006150000861412
:1006800000008610000006140000000006100000A4
:100690000000061100000000080003309E002A0838
:1006A000A200221D061122190615861400008610CC
:1006B0000000A20D9E0B512B08309E002908A200BD
:1006C000A21F0611A21B061586140000861000004A
:1006D000A20D9E0B602B07309E002808A200A20DE1
:1006E000A21F0611A21B061586140000861000002A
:1006F000A20D9E0B702B06118614000086100000C0
:10070000061100000614000000000610000006118B
:10071000000000000800A030A300C830A400A40B13
:100720008F2BA30B8D2B0800FF30A000FF309F0004
:100730009F0B982BA00B962B08000E30A000323098
:0C0740009F009F0BA12BA00B9F2B08001B
:084000000100020009000500A7
:02400E00F13F80
:104200000100D900100002000400000000000000BE
:10421000000000000500BC003000030005000000A5
:10422000000000000000000000000000000000008E
:10423000000000000000000000000000000000007E
:10424000000000000000000000000000000000006E
:10425000000000000000000000000000000000005E
:10426000000000000000000000000000000000004E
:10427000000000000000000000000000000000003E
:00000001FF
